:100000004129A0007F39201B803C0920A01B003C17
:1000100008008A01820700340334063409340C34A2
:1000200010341334163419341C341F34223425345C
:1000300028342B342E3431343334363439343C3490
:100040003F3441344434473449344C344E345134D1
:100050005334553458345A345C345E34603462342A
:100060006434663468346A346B346D346F3470349D
:1000700071347334743475347634783479347A3432
:100080007A347B347C347D347D347E347E347E34EB
:100090007F347F347F347F34A4002508A402031CFE
:1000A000A5032708A602031CA7033709A2003509E8
:1000B000A300A20A0319A30A4130A900AC01AD01B3
:1000C000AE01AF01A8013608840034098E208413E4
:1000D0003D212408AC070318AD0A2508AD07260802
:1000E000AE070318AF0A2708AF072D080120803E8E
:1000F000A1002F080120803EA107210CA8070008BD
:100100003404031C34068000290303194130A9007C
:100110000319A20A0319A30F68283C298417800534
:100120003C299620B4000408B6000800A800053059
:10013000A8190530840000308A0028080739820792
:100140000134023404340834103420344034803410
:100150000F39A0000310A00DA00D1F08E0392004E6
:1001600001389F000030A1003230DD209F149F181D
:10017000B7281E08A10083161E083C2983169B0081
:100180001C141A083C2983169A001C1555309D0032
:10019000AA309D009C149C18CB281C113C29A3015B
:1001A000A200FF30A207031CA307031C3C29033055
:1001B000A100E630DD20D128A101FC3EA000A1096C
:1001C000031CE828FF300000A0070318E328A0075D
:1001D0000000A10FE22808000310A00DA10DFF3EB2
:1001E0000318EC2820083C290310A10CA00CFF3EAA
:1001F0000318F42820083C29A101A301A200033020
:100200000B29A101A301A20001300B29A101A30127
:10021000A20006300B29A80023082102031D122981
:100220002208200204300318013003190230280587
:10023000031DFF303C290038031DFF300405031D5A
:10024000FF303C290404031DFF303C291030A80076
:10025000A101A001A70CA60C031C34292208A007A9
:1002600023080318230FA107A10CA00CA50CA40CB4
:10027000A80B2A2924083C298313031383120000A6
:10028000080089309F00EA01FE30BE20EB00FF30FD
:10029000BE20E800E6010230A820DB002108DC00D7
:1002A0005B08A0005C08A100A30125300321DD004C
:1002B0005B08A0005C08A100A3016E300821DF00EC
:1002C0005D0884005F081B21DF00E0005F08600418
:1002D000031982296B08003C031D71290130EB00D2
:1002E00076296B08013C031D7629EB010030912033
:1002F000E830B7000330B5000630A700A500A430F1
:10030000A6004C205B08A0005C08A1000130A300FF
:1003100000300321DD005B08A0005C08A100013073
:10032000A30049300821DF005D0884005F081B211D
:10033000DF00E0005F0860040319C829FE30BE201A
:10034000EF006F08003C031DAE290130EF0083165B
:10035000FE309B0083126F08C320B9296F08013C4F
:10036000031DB929EF018316FE309B0083126F082D
:10037000C320FE30BE20EB0000309120E830B700F3
:100380000330B5000630A700A500A430A6004C201D
:100390005B08A0005C08A100A3016E300321DD0012
:1003A0005B08A0005C08A100A301B6300821DF00B3
:1003B0005D0884005F081B21DF00E0005F08600427
:1003C00003190D2AFF30BE20EF006F084B3C031DC0
:1003D000F2297830EF008316FF309B0083126F08FC
:1003E000C320FE296F08783C031DFE294B30EF0027
:1003F0008316FF309B0083126F08C320FF30BE209E
:10040000E80000309120E830B7000330B500063036
:10041000A700A500A430A6004C200230A820DB00D5
:100420002108DC000A30CF205B08A0005C08A10096
:10043000A30125300321031D0D2A0130ED006B08B7
:10044000003C031D242AB8016B08013C031D2A2A25
:100450000E30B800FF30B9000230A820DB002108C0
:10046000DC00E7015B08A0005C08A100A3012530C7
:100470000821031D3C2A49220A30CF20E60A6608DB
:10048000FA3C031D482A0510831605108312E60165
:100490002C2A5B08A0005C08A1000330A300923066
:1004A0000321DD005B08A0005C08A1000330A3006D
:1004B000FF300821DF005D0884005F081B21DF009A
:1004C000E0005F0860040319692A0130E300EF24AB
:1004D0003A245B08A0005C08A1000330A300493067
:1004E0000321DD005B08A0005C08A1000330A3002D
:1004F00092300821DF005D0884005F081B21DF00C7
:10050000E0005F0860040319892A0230E300EF2449
:100510003A245B08A0005C08A1000230A300FF3071
:100520000321DD005B08A0005C08A1000330A300EC
:1005300049300821DF005D0884005F081B21DF00CF
:10054000E0005F0860040319A92A0330E300EF24E8
:100550003A245B08A0005C08A1000230A300B6307A
:100560000321DD005B08A0005C08A1000230A300AD
:10057000FF300821DF005D0884005F081B21DF00D9
:10058000E0005F0860040319C92A0430E300EF2487
:100590003A245B08A0005C08A1000230A3006D3083
:1005A0000321DD005B08A0005C08A1000230A3006D
:1005B000B6300821DF005D0884005F081B21DF00E2
:1005C000E0005F0860040319E92A0530E300EF2426
:1005D0003A245B08A0005C08A1000230A30025308B
:1005E0000321DD005B08A0005C08A1000230A3002D
:1005F0006D300821DF005D0884005F081B21DF00EB
:10060000E0005F0860040319092B0630E300EF24C3
:100610003A245B08A0005C08A1000130A300DB3095
:100620000321DD005B08A0005C08A1000230A300EC
:1006300025300821DF005D0884005F081B21DF00F2
:10064000E0005F0860040319292B0730E300EF2462
:100650003A245B08A0005C08A1000130A30091309F
:100660000321DD005B08A0005C08A1000130A300AD
:10067000DB300821DF005D0884005F081B21DF00FC
:10068000E0005F0860040319492B0830E300EF2401
:100690003A245B08A0005C08A1000130A3004930A7
:1006A0000321DD005B08A0005C08A1000130A3006D
:1006B00091300821DF005D0884005F081B21DF0006
:1006C000E0005F0860040319692B0930E300EF24A0
:1006D0003A245B08A0005C08A1000130A3000030B0
:1006E0000321DD005B08A0005C08A1000130A3002D
:1006F00049300821DF005D0884005F081B21DF000E
:10070000E0005F0860040319892B0A30E300EF243E
:100710003A245B08A0005C08A100A301B6300321C5
:10072000DD005B08A0005C08A1000130A3000030E0
:100730000821DF005D0884005F081B21DF00E00066
:100740005F0860040319A82B0B30E300EF243A2460
:100750005B08A0005C08A100A3016E300321DD004E
:100760005B08A0005C08A100A301B6300821DF00EF
:100770005D0884005F081B21DF00E0005F08600463
:100780000319C62B0C30E300EF243A245B08A000C9
:100790005C08A100A30125300321DD005B08A00057
:1007A0005C08A100A3016E300821DF005D08840011
:1007B0005F081B21DF00E0005F0860040319E42BE1
:1007C0000D30E300EF243A240230A820DB0021089A
:1007D000DC00E70A6708A00064300121DD005B0847
:1007E000A0005C08A100A30125300321DF005D0803
:1007F00084005F081B21DF00E0005B08A0005C08AC
:10080000A100A3016E300821E1005F0860048400AC
:1008100061081B21E100E200610862040319112C48
:100820004B276A08003C031D2D2C6708A000C83028
:100830000121DD005B08A0005C08A100A3016E306F
:100840000321DF005D0884005F081B21DF00E0005A
:100850005F08600403192D2C5D240A30CF205B084B
:10086000A0005C08A100A30125300321031DE42B97
:10087000E60108006D08223C031DFF30FF3ADD0051
:100880006A08013C031DFF30FF3ADF005D08840069
:100890005F082221DF00E0005F0860040319512C8B
:1008A00008006D08383E840063088000ED0A6D087A
:1008B000383E8400FF3080000800FF306D07DD0007
:1008C000FF300318013EDE005D08383E8400FF3033
:1008D0008000ED010730630203187E2CFF306307B0
:1008E000DD00FF300318013EDE002230A600A70124
:1008F0005D08A2005E08A3002621F0006308A000A6
:100900000730FC20DD006308A0000C300621DF006A
:100910005D0884005F081B21DF00E0005F086004C1
:100920000319A22CF9306307DD00FF300318013EE4
:10093000DE002230A600A7015D08A2005E08A30029
:100940002621F0006D08383E84000008DD005D08B7
:10095000FF3C031DE02C0F30E400A927700883162C
:100960009B0083126408C3200130ED006B08003C3B
:10097000031DBB2CB8016B08013C031DC12C0E30BC
:10098000B800FF30B90000309120E830B7000330E4
:10099000B5000530A700A500DC30A6004C200230D1
:1009A000A820DB002108DC000A30CF205B08A00073
:1009B0005C08A100A30125300321031DCF2C0800F2
:1009C0006D08383E84000008E400A92770088316EB
:1009D0009B0083126408C320ED0AF00AA22C6A0867
:1009E000003C031DF42C472D6308A0000130FC20BF
:1009F000DD006308A00006300621DF005D088400EA
:100A00005F081B21DF00E0005F0860040319182D58
:100A1000FF306307DD00FF300318013EDE002230A7
:100A2000A600A7015D08A2005E08A3002621EE0033
:100A30006308A0000730FC20DD006308A0000C3034
:100A40000621DF005D0884005F081B21DF00E00055
:100A50005F08600403193C2DF9306307DD00FF30A7
:100A60000318013EDE002230A600A7015D08A200A7
:100A70005E08A3002621EE000D306302031C412D09
:100A800008006308E5006E08BE20E400C2276B087A
:100A9000013C03193B2E63080F3C031D502D080039
:100AA0006308003C031D552DEB016308013C031D49
:100AB000662D003091206808B700B5018430A6008B
:100AC0000330A7000230A500BC304C206308023C74
:100AD000031D772D003091206808B700B5014C3018
:100AE000A6000430A7000230A500BC304C206308EB
:100AF000033C031D882D003091206808B700B50124
:100B00004C30A6000430A7000330A50084304C20F0
:100B10006308043C031D992D003091206808B7003C
:100B2000B5011430A6000530A7000230A500BC3086
:100B30004C206308053C031DAA2D00309120680855
:100B4000B700B5011430A6000530A7000330A5009A
:100B500084304C206308063C031DBB2D00309120DF
:100B60006808B700B5011430A6000530A7000430AE
:100B7000A5004C304C206308073C031DCC2D0030F1
:100B800091206808B700B501DC30A6000530A70049
:100B90000230A500BC304C206308083C031DDD2D4D
:100BA000003091206808B700B501DC30A6000530A0
:100BB000A7000330A50084304C206308093C031DC6
:100BC000EE2D003091206808B700B501DC30A6009A
:100BD0000530A7000430A5004C304C2063080A3CC7
:100BE000031DFF2D003091207830B700B501A430EF
:100BF000A6000630A7000430A5004C304C20630846
:100C00000B3C031D102E003091206808B700B50181
:100C1000DC30A6000530A7000530A50014304C20BC
:100C200063080C3C031D212E003091206808B7009A
:100C3000B501A430A6000630A7000530A500DC30C1
:100C40004C2063080D3C031D312E00309120E8300C
:100C5000B7000330B5000A30A700A5002830A60071
:100C60004C2063080E3C031D372E0130EB006B084F
:100C7000003C0319272F63080F3C031D402E08007A
:100C80006308003C031D452EEB016308013C031D76
:100C9000562E003091206808B700B501B930A60083
:100CA0000430A7000230A500B9304C206308023C94
:100CB000031D672E003091206808B700B501383059
:100CC000A6000530A7000230A500B9304C2063080B
:100CD000033C031D782E003091206808B700B50151
:100CE000C530A6000530A7000230A500B9304C2061
:100CF0006308043C031D892E003091206808B7006A
:100D0000B501B930A6000430A7000330A5000230B9
:100D10004C206308053C031D9A2E00309120680882
:100D2000B700B5013830A6000530A7000330A50094
:100D300002304C206308063C031DAB2E003091208E
:100D40006808B700B501C530A6000530A70003301C
:100D5000A50002304C206308073C031DBC2E003068
:100D600091206808B700B501B930A6000430A7008B
:100D70000330A50054304C206308083C031DCD2EE1
:100D8000003091206808B700B5013830A600053062
:100D9000A7000330A50054304C206308093C031D14
:100DA000DE2E003091206808B700B501C530A600DE
:100DB0000530A7000330A50054304C2063080A3CDE
:100DC000031DEF2E003091206808B700B501B9303F
:100DD000A6000430A7000330A500AD304C20630806
:100DE0000B3C031D002F003091206808B700B501AF
:100DF0003830A6000530A7000330A500AD304C20E8
:100E000063080C3C031D112F003091206808B700C7
:100E1000B501C530A6000530A7000330A500AD30F0
:100E20004C2063080D3C031D212F00309120E83039
:100E3000B7000330B5000A30A700A5002830A6008F
:100E40004C2063080E3C031D272F0130EB00630884
:100E50000D3C031DFF30FF3ADD006A08013C031D15
:100E6000FF30FF3ADF005D0884005F081B21DF00D0
:100E7000E0005F0860040319412F0530A300DC3057
:100E8000D0206A08003C031D462F0800EE0A6808BF
:100E9000CF20432D08006A08013C031D6A2FEA0198
:100EA0006C08EB00E701003091204B30B700B50132
:100EB0000630A700A500A430A6004C2000309120E9
:100EC0004B30B700B5010530A700A5001430A600CF
:100ED0004C20982F6A08003C031D982F0130EA002F
:100EE0006B08EC00E701003091204B30B700B501F2
:100EF0000530A700A5001430A6004C20003091203A
:100F00004B30B700B5010630A700A500A430A600FD
:100F10004C200130ED006B08003C031D902FB80100
:100F20006B08013C031D962F0E30B800FF30B9004E
:100F30000230A820DB002108DC000A30CF205B084B
:100F4000A0005C08A100A30125300321031D982FF8
:100F5000080007306302031CB42F0F30E900640857
:100F6000A0000430EF20E400073063020318BA2F1A
:100F7000F030E9007008BE20EF006908EF056F0847
:100F8000E40408006508A0000730FC20DD006508C7
:100F9000A0000C300621DF005D0884005F081B21E3
:100FA000DF00E0005F0860040319DD2F6408A00083
:100FB000A1010430F720E300F62F6508A0000130FE
:100FC000FC20DD006508A00006300621DF005D087A
:100FD00084005F081B21DF00E0005F086004031944
:0E0FE000F62F0F30E90064086905E3000800F1
:02400E00E2309E
:02420000FF00BD
:02424400FF0079
:02428800FF0035
:0242CC00FF00F1
:02431000FF00AC
:02435400FF0068
:0443FC0000004B0072
:00000001FF
